:020000020000FC
:100000000C942E000C942E000C9492010C94FF0181
:100010000C942E000C945B020C942E000C942E0079
:100020000C942E000C942E000C942E000C942E0098
:100030000C942E000C942E000C942E000C942E0088
:100040000C942E000C942E000C942E000C942E0078
:100050000C942E000C942E000C940A02F89404E0E8
:100060000EBF0FEF0DBF2224B1E0A0E02D92B23001
:10007000E9F700E01FEF04B915B908E010E00DB989
:100080001EB904E01EEF00BB11BB08E110E003BB8A
:1000900014BB00E80093610004E0009361000EE0EF
:1000A0000093640005EA0093E50003E00093E60096
:1000B0000CEE0093E70008EC0093E40073E002E428
:1000C00000937C0003E100937A000BE700937E002D
:1000D00003E00093B00001E00093700008E000939B
:1000E000B60002E000936B0001EF00936C0000EC9F
:1000F0000DBB2EBA2ABC772409E00093290100E049
:1001000010E0DBD50F3F11F0B9D58EC005E01EE140
:10011000009300021093010206E01EE10093080222
:100120001093090200931002109311020093180219
:1001300010931902009320021093210200E010E0B6
:100140000093280210932902009330021093310289
:1001500002E110E0009302021093030200930A02EE
:1001600010930B02009312021093130200931A02D1
:1001700010931B02009322021093230200E010E070
:1001800000932A0210932B02009332021093330241
:1001900000E010E0009304021093050200930C02AB
:1001A00010930D02009314021093150200931C0289
:1001B00010931D02009324021093250200E010E02A
:1001C00000932C0210932D020093340210933502F9
:1001D00000E010E0009306021093070200930E0265
:1001E00010930F02009316021093170200931E0241
:1001F00010931F02009326021093270200E010E0E4
:1002000000932E0210932F020093360210933802AF
:1002100001EE10E00093390210933A0204EB10E073
:1002200000933B0210933C027894F49A00913902B7
:100230000093200100913A020093210102E0009313
:10024000220101E0009336010E94CE0A0E94690B50
:1002500093D2F499F9CFE7D118D36FD30E94940ABF
:10026000AAD53ED5BCD1F79903C022D20E94490A33
:100270000AB500FD41C001FD47C005FD47C0009122
:100280002201013031F1033039F1043041F1003005
:1002900049F1023049F10530C9F00630A1F00730CC
:1002A00079F0083051F0093029F00A3009F030C0F7
:1002B000A8D72EC00E945B092BC00E94810928C0CC
:1002C0000E94A70925C00E94C70922C00E94E70911
:1002D0001FC00E94FF091CC00E941B0A19C00E9477
:1002E000320A16C03BD714C00091240102FF02C09D
:1002F0005ED70EC07DD60CC071FCC1CF0091240129
:100300000770003009F0BBCF2CD602C095D500C0D5
:100310000E947C0B0E942B0C07E003BF889506E02F
:1003200003BF92CFF39B1895BFB6BF920F931F9355
:100330002F93F29B03C0619904C05BC0619B01C015
:1003400058C000912F01033021F0039500932F0135
:1003500044C00091B20010911C0100931C01011BCC
:1003600000932B018A9599F480E11091440120912A
:100370004501269517952695179526951795269547
:10038000179510934301209244012092450110914A
:10039000440120914501100F221D10934401209328
:1003A000450120921901F2990BC00091140110919E
:1003B000150101501209009314011093150119C081
:1003C0000091140110911501BB24B3940B0D121D63
:1003D00000931401109315010CC00091B20000931A
:1003E0001C0181E1209244012092450120924301A9
:1003F000D8CF2F911F910F91BF90BFBE1895BFB658
:10040000BF920F9308EC0093E40073E00F91BF904C
:10041000BFBE1895BFB6BF920F931F9303B100954F
:10042000017F003061F4533020F0523310F4F59A1C
:1004300002C000931A01552700931B0133C010918D
:100440001B01011721F0552700931B012BC00093BE
:100450001B015F3F21F05395533008F427C00093F0
:100460001A01003119F0013009F016C000913D0168
:100470000F3F31F0039500933D01093108F416C098
:1004800000911D01039500931D01083009F00EC075
:1004900020921D01F59A0AC0523341F400931A01CB
:1004A000F59A04C020923D0120921D011F910F91E9
:1004B000BF90BFBE1895BFB6BF920F931F932F93E7
:1004C000F19B27C000914301109116011330B9F43C
:1004D0001AB516FDA1F010914201103081F023E011
:1004E000120F011760F01AB510641ABD112710938E
:1004F000150112E31093140106E00093EC00109133
:100500002D01F49B10912E01101718F401E00093B7
:100510001901009119010F3F99F0039500931901FA
:10052000023019F0043019F00BC0F19809C0F398AB
:100530007398F49B05C00091160103950093160172
:1005400004E07394701609F044C0772400912401EC
:10055000039500932401662319F06A9509F4F69A2D
:10056000F49B20C000912C010030E1F00A9500932B
:100570002C01C1F40091430100934201102F169504
:1005800016951695010F08F40FEF015000932D01F9
:10059000010F08F40FEF015000932E0102E00093C9
:1005A000EC0017C0009123010A950093230151F438
:1005B00004EB009323018A9A00000000000003EC82
:1005C00000937A00703029F07A9519F400EC0093CA
:1005D000E4002F911F910F91BF90BFBE189500911D
:1005E00024010030F9F400912A010630D9F4009179
:1005F00026010A30B9F400912501003099F4F49AEB
:100600000AB504600ABD0091F1000E7F0093F1006D
:100610000091F6000E7F0093F6000091EC000E7F33
:100620000093EC000895F79908950091240100309B
:1006300009F00895A0E0B2E000912A01000F000F38
:10064000000FA00FB21D1D910D91D0902601C090FA
:1006500025010C151D0521F4009134010E94050CA3
:100660001D910D91D0902601C09025010C151D05FE
:1006700021F4009134010E94180C1D910D91D0902D
:100680002601C09025010C151D0521F400913401AF
:100690000E94050C1D910D91D0902601C09025015E
:1006A0000C151D0521F4009134010E94180C0895C9
:1006B0000AB505FD0895A0E0B2E0009135010030D3
:1006C00039F0035006950695000F000F000F05C086
:1006D00000912A01000F000F000FA00FB21D0C9116
:1006E00012961C91101BCC24DD24EE2428E1201B43
:1006F000112341F00894E794D794C7942A9511F0F8
:100700001A95B1F7222331F08894E794D794C794CF
:100710002A95C1F7E0923A01D0923901C09238018E
:1007200012960C9112961C91101BCC24DD24EE2401
:1007300028E1201B112341F00894E794D794C79433
:100740002A9511F01A95B1F7222331F08894E79495
:10075000D794C7942A95C1F70091380110913901B7
:1007600020913A010C291D292E290093380110935C
:10077000390120933A0108957210089500912401DF
:100780000C33B1F4209224010091250103950093CC
:10079000250100913201003059F00A950093320191
:1007A00039F4009134010D7F009334010E94E20B73
:1007B000009125010C3359F5209225010091260165
:1007C0000395009326010AB503FD21C0009127017E
:1007D0000831E8F000912A010630C9F4009128019F
:1007E000093019F0023049F012C00091260103309F
:1007F00071F40A950093260107C00091260102308A
:1008000031F40395009326010AB508600ABD0091F2
:100810002601083199F40AB5077F0ABD2092260106
:100820000091270103950093270100912A01039568
:1008300000932A01073011F420922A010091280127
:10084000E0E2FCE1E00FF21D149100912901037038
:1008500029F400912801013009F413950091270132
:10086000011739F420922701009128010395009384
:100870002801009128010C3039F4209228010091C0
:100880002901039500932901089500917A0004FF3E
:100890000895037900937A0000917C00023429F0D6
:1008A000003491F00E3519F10895009178001091FF
:1008B0007900009353011093540100E400937C00ED
:1008C00003ED00937A0008958A98009178001091C2
:1008D000790000930201109303010EE500937C0060
:1008E00003ED00937A000AB500610ABD08950091F6
:1008F000780010917900009311011093120102E425
:1009000000937C0000E100937A0001D008950091EB
:1009100011011091120121E0003F120728F421E09B
:10092000003C120730F408950AB502600E7F0ABD3C
:1009300008950AB501600ABD08950AB504FF089537
:10094000109124011A3308F008950F7E0ABD00911A
:1009500002011091030120EE822E2EE2922E2091B0
:10096000530130915401201B310B199D7001089DDA
:100970006001189DD00CE11CF21C909ED00CE11C73
:10098000F21C41E000271127C21AD30AE208F2083C
:1009900018F0040F121DF8CFFBE1EAEE42E32EEC53
:1009A000C22E2FEFD22E259135912030320541F104
:1009B0002017310728F0E22EF32EC40ED21CF3CFFD
:1009C000EF92FF92E21AF30A21E0822E22273327C8
:1009D000E41AF20818F0280D321DFACF41E0FF901A
:1009E000EF90E21AF30AE016F1061CF0C40ED21CD6
:1009F000F8CFC0920001D0920101F49B05D0089578
:100A00000FEFC02ED02EF5CFC0901701D090180157
:100A10000AB501FF08C006E4C01AD208C0921E0140
:100A2000D0921F0108950091000110910101C09022
:100A30002001D0902101C01AD10A860110F40027AC
:100A40001127009351011093520100914801109118
:100A500049010C0D1D1D12F40027112720913E01A4
:100A600030913F01369527950217130708F0890149
:100A7000009348011093490116950795C0905101C4
:100A8000D0905201CC0CDD1CCC0CDD1CCC0CDD1C40
:100A9000CC0CDD1C0C0D1D1D00934601109347016D
:100AA000209117013091180124513209201B310B7C
:100AB00018F02233320510F422E330E0F399089560
:100AC00020931E0130931F010895FBE1EEEB0053CC
:100AD000E00FF21D8490982C2FE0822220EF9222CA
:100AE0009294103049F01130D1F0123019F01330D7
:100AF00011F0089533C045C0880C880C880C990CFF
:100B0000990C990C0091F100077808290093F100E5
:100B10000091F600077A09290093F6000895AA24A7
:100B20008694A7940091F1000F770A290093F100B1
:100B30000091F200087F08290093F200AA249694FD
:100B4000A7940091F6000F770A290093F600009110
:100B5000F7000A7F09290093F7000895880C880C94
:100B6000880C990C990C990C0091F20007780829CF
:100B70000093F2000091F700077A09290093F7002B
:100B80000895AA248694A7940091F2000F770A2969
:100B90000093F2000091F300087F08290093F3000E
:100BA000AA249694A7940091F7000F770A2900933E
:100BB000F7000091F8000A7F09290093F8000895D2
:100BC000CC24DD24EE24FF24083E23E0120720F08D
:100BD000085E1340F394F8CF043620E0120720F0AB
:100BE00004561040E394F8CF0A3018F00A50D3941A
:100BF000FBCFC02E00E3F00EE00ED00EC00E089525
:100C0000102F107F1295D12E10E3D10E1AE3D116BA
:100C100010F017E0D10E102F1F70C12E10E3C10E7F
:100C20001AE3C11610F017E0C10E089500912801D3
:100C3000E4E1FCE1E00FF21DC0902701C394D490E1
:100C4000E090290100912801023008F4EA94CD0CCB
:100C5000CE0CE694E69404E106950695CE0CC00E03
:100C600004E6C00E07E0C01610F0C01AFCCF0C2D31
:100C7000015008F406E000932A010895A0E0B2E0D4
:100C8000C0E0D0E03CE38E0118D00D9321963A9558
:100C9000D1F70895A0E0B2E0C0E0D0E03CE30D91D0
:100CA000C02E8E010AD0C01621F00C2D2D2F1C2F26
:100CB0000DD021963A9599F70895F999FECFF894B9
:100CC00012BD01BDF89A00B578940895F999FECF48
:100CD000F89422BD11BD00BDFA9AF99A789408954E
:100CE0000091F6000B7FF79904600093F6000AB5B7
:100CF00005FD07C00091F1000D7FF79B0260009396
:100D0000F100009136010370003029F0013049F004
:100D1000023069F014C00091F3000F7E0093F300DD
:100D20000EC00091F30000610093F30008C0009131
:100D3000F3000F7E70FE00610093F30000C000918D
:100D400036010C70003029F0043049F0083069F0A9
:100D500014C00091F8000F7E0093F8000EC00091BF
:100D6000F80000610093F80008C00091F8000F7EC1
:100D700070FE00610093F80000C00091360100731E
:100D8000003029F0003149F0003269F008950091F7
:100D9000F300077F0093F30008950091F3000860CB
:100DA0000093F30008950091F300077F70FE086040
:100DB0000093F3000895F69B0AC0F3996BDFF69851
:100DC00002E00093220100E000933501A6D30091D8
:100DD0003501003009F008950091340101FD28C06B
:100DE00000FF02C013C0089500912001109121015D
:100DF000C0903902D0903A020C151D0511F401E0A3
:100E000002C000E000C00093360108950091200167
:100E100010912101C0903B02D0903C020C151D05A1
:100E200011F404E002C000E000C000933601089510
:100E300000E100933601089500913301003079F00C
:100E4000013079F0023079F0033079F0043079F034
:100E5000053079F0063079F02092330108953ED0C4
:100E6000089568D0089551D1089578D1089502D198
:100E7000089515D108958CD008950091240107702C
:100E80000030F9F0C0901701D090180100913E0198
:100E900010913F01D694C7943EE30C191D0918F434
:100EA0003CE3019511278CDE0EE310E00EDE032FEC
:100EB00011E00BDE0D2D12E008DE0C2D13E005DE37
:100EC000089500E510E001DE0FE411E0FEDD06E428
:100ED00012E0FBDD03E513E0F8DD089506E410E021
:100EE000F4DD08E06DDE0E2D11E0EFDD0D2D12E0DA
:100EF000ECDD0C2D13E0E9DD0091F60001600093BC
:100F0000F6000895009147017BDE0D2D10E0DDDD38
:100F10000C2D11E0DADD0091460172DE0D2D12E09C
:100F2000D4DD0C2D13E0D1DD0091F6000E7F00938F
:100F3000F6000895109147010091460141DE0F2D02
:100F400010E0C3DD0E2D11E0C0DD0D2D12E0BDDD82
:100F50000C2D13E0BADD0091F6000E7F0093F60031
:100F6000089502E410E0B1DD01E411E0AEDD04E536
:100F700012E0ABDD04E513E0A8DD0091F1000E7F87
:100F80000093F1000091F6000E7F0093F6000895A3
:100F90000091120135DE0D2D10E097DD0C2D11E0D2
:100FA00094DD009111012CDE0D2D12E08EDD0C2D53
:100FB00013E08BDD0091F6000E7F0093F60008959C
:100FC000009103011DDE0D2D10E07FDD0C2D11E0E1
:100FD0007CDD0091020114DE0D2D12E076DD0C2D7A
:100FE00013E073DD0091F6000E7F0093F600089584
:100FF000009126011127E4DD0D2D003309F40EE3E5
:1010000010E063DD0C2D11E060DD0091250111275A
:10101000D7DD0D2D12E059DD0C2D13E056DD0091CA
:10102000F6000E7F71FC01600093F6000091F10064
:101030000E7F71FC01600093F1000091EC000160F3
:101040000093EC000895052FDBDD0D2D10E03DDD54
:101050000C2D11E03ADD00911A01D2DD0D2D12E0C8
:1010600034DD0C2D13E031DD0091F6000E7F00938E
:10107000F600089500914201C3DD06E410E025DD8D
:1010800002E511E022DD0D2D12E01FDD0C2D13E035
:101090001CDD0091F6000E7F0093F600089500918C
:1010A0004301AEDD0D2D10E010DD0C2D11E00DDD46
:1010B00000911901A5DD0D2D12E007DD0C2D13E0C7
:1010C00004DD0091F60001600093F6000091F1004C
:1010D0000E7F639901600093F1000895109115014E
:1010E000009114016DDD0F2D10E0EFDC0E2D11E0ED
:1010F000ECDC0D2D12E0E9DC0C2D13E0E6DC0091B8
:10110000F6000E7F0093F600089500912401077009
:101110000030B9F0109115010091140151DD0F2D2F
:1011200010E0D3DC0E2D11E0D0DC0D2D12E0CDDC73
:101130000C2D13E0CADC0091F6000E7F0093F60040
:10114000089502E510E0C1DC06E411E0BEDC0CE429
:1011500012E0BBDC03E413E0B8DC08950091240145
:1011600007700030B9F010911F0100911E0128DDB9
:101170000F2D10E0AADC0E2D11E0A7DC0D2D12E0E2
:10118000A4DC0C2D13E0A1DC0091F6000E7F00938F
:10119000F600089500E510E098DC0FE411E095DC1E
:1011A00003E512E092DC09E413E08FDC089500917E
:1011B0000001109101010F3F39F41F3F29F40CE3A6
:1011C000E02ED02EC02E01C0FBDC0E2D10E07DDC09
:1011D0000D2D11E07ADC0C2D12E077DC0AE313E030
:1011E00074DC0091F60001600093F6000091F100BC
:1011F0000E7F0093F1000091EC0001600093EC0081
:10120000089500912401037019F471FE01C035C0E6
:10121000A0E0B2E0009135010350A00FA00FB21D75
:101220000D911127CDDC0D2D10E0003309F40EE3F4
:101230004CDC0C2D11E049DC0C911127C1DC0D2D8B
:1012400012E043DC0C2D13E040DC0091F100016062
:101250000093F1000091F60001600093F600009108
:10126000F10004600093F10000913501035011E09A
:1012700000FD14E0109336010895009135010350EC
:101280000695332700FD31E006950395112798DC7C
:101290000C2D11E01ADC00E510E017DC032F0F5CC9
:1012A00012E013DC0EE313E010DC0091F1000E7F7E
:1012B0000093F100D9CF00912501112781DC0EE3C5
:1012C00070FE0D2D12E001DC0EE370FE0C2D13E01C
:1012D000FCDB00912601112773DC0D2D003309F48E
:1012E0000EE310E0F2DB0C2D11E0EFDB0091F100DA
:1012F00001600093F1000091F60001600093F60098
:1013000008950091260111275BDC0EE370FE0D2D80
:10131000003309F40EE310E0D8DB0EE370FE0C2D71
:1013200011E0D3DB0091250111274ADC0D2D12E0DD
:10133000CCDB0C2D13E0C9DB0091F10001600093C0
:10134000F1000091F60001600093F600089500910D
:1013500027010395112734DC0EE370FE0D2D10E0FC
:10136000B4DB0EE370FE0C2D11E0AFDB0091280121
:101370000395112725DC0D2D12E0A7DB0C2D13E0C2
:10138000A4DB0091F60001600093F600089500913F
:1013900028010395112714DC0EE370FE0D2D12E0D9
:1013A00094DB0EE370FE0C2D13E08FDB0091270120
:1013B0000395112705DC0D2D10E087DB0C2D11E0C6
:1013C00084DB0091F60001600093F60008952091FF
:1013D000290100ED17E0020F121DF2DB0F2D10E0C6
:1013E00074DB0E2D11E071DB0EE370FE0D2D12E0AB
:1013F0006CDB0EE370FE0C2D13E067DB08950091AB
:10140000200110912101DCDB0E2D10E05EDB0D2DA3
:1014100011E05BDB0C2D12E058DB0AE313E055DB37
:101420000091F1000E7F0093F1000091F600016041
:101430000093F60008950091390210913A02C0DB42
:101440000E2D10E042DB0D2D11E03FDB0C2D12E0E4
:101450003CDB0AE313E039DB0091F6000160009306
:10146000F600089500913B0210913C02A9DB0E2D7D
:1014700010E02BDB0D2D11E028DB0C2D12E025DB1D
:101480000AE313E022DB0091F60001600093F6000E
:1014900008950AB505FD0895009138011091EC00FA
:1014A00007FB000F1170102B1093EC000091390115
:1014B000112710F900FB11F901FB12F906FB13F9D2
:1014C00007FB14F92091F7002D7D02FB21F905FBA4
:1014D00025F92093F7002091F6002F7D03FB25F9D5
:1014E0002093F6002091F8002D7F04FB21F9209332
:1014F000F80000913A0100FB15F901FB16F902FB17
:1015000017F91093ED001091EE00107E06950695E8
:101510000695102B1093EE000895ACEEBB272D928C
:10152000AE3FE9F72C92089500911E0110911F0122
:1015300020911401309115012017310709F142E083
:10154000041B12092017310788F044E0040F121D14
:101550000217130708F00895F3990895F298F19A85
:10156000739A20922B0120922F010895F3990895E8
:10157000F29AF19A739A20922B0120922F010895EA
:10158000F19B0895F198209219010AB501FF089581
:10159000A498A3982092700073980895F49B0895DE
:1015A00073E000911601003031F0023021F1043077
:1015B00009F0089569C0F39908950DE310E085DA04
:1015C0000DE311E082DA0DE312E07FDA0DE313E0C0
:1015D0007CDA00911601039500931601F298F19AB6
:1015E000739A20922B0120922F0100ED00932D0180
:1015F00000932E010895F39908950FE410E065DA41
:1016000000E511E062DA05E412E05FDA0EE413E0CF
:101610005CDA0AB502FD11C010911A01103499F577
:1016200001E410E052DA04E411E04FDA01E412E0E0
:101630004CDA00E513E049DA0CC004E410E045DAC6
:1016400005E411E042DA03E512E03FDA03E413E0D7
:101650003CDA11270AE00093140110931501009160
:10166000160103950093160120922B0120922F0161
:1016700005E000932C010AB50F7B0ABD20924201C0
:10168000F29AF19A739A0895F399089500911401CA
:1016900010911501009317011093180116950795E5
:1016A00000933E0110933F012AB522FF03C02B7F18
:1016B0002ABD0BC000913E0110913F0100931E0115
:1016C00010931F0101E00093230120921601F4986A
:1016D0000895F19903C0A498A3980895F29B06C0B9
:1016E000A49800000000A39AF39A0895A39800001C
:1016F0000000A49AF39A0895F59B089573E0F59875
:1017000000911A01003199F0013059F00032A9F02E
:10171000003429F0003861F1013111F0089547C01B
:1017200093C000913B01016000933B01089500913B
:101730003B01026000933B010895523311F40FE125
:1017400009C0009135010395043221F402E00093B1
:10175000220100E00093350100913B0104600093F9
:101760003B01DBDE00913601007F009336010895D6
:1017700000913501003009F00895523381F00AB527
:1017800005FF07C000913301039500933301C5DEC7
:10179000089510E80EB301270EBBBFDE08950AB509
:1017A00010E201270ABDB9DE2092330108950091AD
:1017B0003501003009F0089500913401523319F5D4
:1017C00001FF0CC00D7F0093340100914001109186
:1017D0004101009320011093210122C00260009377
:1017E00034010091200110912101009340011093D8
:1017F000410108E710E000932001109321010AE065
:10180000009332010DC000FF13C00E7F009334011E
:101810000091390210913A020093200110932101A6
:101820000AE00093230101E00093220165E008959E
:1018300001600093340100913B0210913C0200933F
:10184000200110932101ECCF523321F466DEF19890
:10185000F398F49A089500913B01003009F408953B
:1018600000913501003011F413D10895013011F4C5
:1018700046D10895023011F472D108950F3111F458
:10188000E7D00895003211F444D00895013211F4E4
:1018900060D00895023211F49CD00895033211F4FF
:1018A000B7D00895033020F0023210F402D008952A
:1018B0000895A0E0B2E0009135010350A00FA00F01
:1018C000B21D00913B0100FD03C001FD16C00EC01A
:1018D0001D910C912AE0020F0C3329F40027139577
:1018E000183109F4112711971D930C930AE0009306
:1018F000220164E120923B0108951D910C912AE0A0
:10190000021B063F81F702E31A951F3F61F717E1BB
:10191000EACF00913B0100FD03C001FD11C008C0EA
:101920000091280103950C3009F400270093280149
:1019300006E0009322016AE020923B0177D90895E6
:10194000009128010A950F3F09F40BE0009328014C
:10195000EFCF00913B0100FD03C001FD20C017C087
:1019600000912801E0E2FCE1E00F149100912901CF
:10197000037029F400912801013009F413950091B6
:1019800027010395011709F400270093270107E0B9
:10199000009322016AE020923B0148D9089500910A
:1019A0002801E0E2FCE1E00F1491009129010370AD
:1019B00029F400912801013009F4139500912701C1
:1019C0000A950F3F11F4012F0A9500932701DFCFED
:1019D000089500913B0100FD03C001FD10C008C047
:1019E000009126010395083109F400270093260190
:1019F00008E0009322016AE020923B0108950091E3
:101A000026010A950F3F09F407E100932601F0CF64
:101A100000913B0100FD03C001FD10C008C0009112
:101A2000250103950C3309F400270093250109E0F3
:101A3000009322016AE020923B0108950091250164
:101A40000A950F3F09F40BE300932501F0CF0895A9
:101A500000913B0100FD03C001FD11C008C00091D1
:101A600029010395043609F409E00093290105E0F2
:101A7000009322016AE020923B01D8D8089500919A
:101A800029010A95083009F403E600932901EFCFF4
:101A900000913B0100FD03C001FD1AC016C001E02A
:101AA0000093220163E0009120011091210121E0C7
:101AB0000039120750F425E0020F121D0093200197
:101AC000109321010AE00093230120923B01089525
:101AD00001E00093220163E00091200110912101B7
:101AE00020E00233120788F325E0021B120900935D
:101AF0002001109321010AE000932301E6CF03E0C7
:101B00000093220100913B0100FD03C001FD17C0BD
:101B10000FC00091390210913A0221E00C321207F5
:101B200038F425E0020F121D0093390210933A0297
:101B300002E0009336016AE020923B010895009193
:101B4000390210913A0220E00436120788F325E0AA
:101B5000021B12090093390210933A02E9CF04E004
:101B60000093220100913B0100FD03C001FD17C05D
:101B70000FC000913B0210913C0220E00A3F120787
:101B800038F425E0020F121D00933B0210933C0233
:101B900008E0009336016AE020923B01089500912D
:101BA0003B0210913C0220E00233120788F325E04B
:101BB000021B120900933B0210933C02E9CFBD883F
:101BC0003EAE8BA7B78CBFAF0F80028A0000009F8C
:101BD000B335BA3717009B88A800310092BD1F8F1C
:101BE00012A733B9B00000AB3E002A85C666D84FB5
:101BF000803E423110272D1F081936146A10670DD8
:101C0000000B1209850743063C056604B50324034F
:101C1000AC0200001C1F0205070A0C0F1214171952
:0C1C20001F1C1F1E1F1E1F1F1E1F1E1F4B
:00000001FF
